:020000040000FA
:100000008B018A018301E228F000030E8301F100D5
:100010000408F3008C1E5828981C18195528181C21
:1000200028284611C5011A08C000C6197128603A6F
:10003000031925284008410603194A28A03A031944
:100040002528603A03193E287128C40146157128F5
:100050002030450784001A08461D71288000C40618
:10006000C50A2030840000080F39023E4506031DF2
:100070007128461144080319C6157128061420304A
:10008000990083160313981C43288312031320300E
:1000900099006628461C71280614831603130C1653
:1000A00083120313C201C6145C281A08181218160A
:1000B0000C1E7128C61C6628A03042078400000868
:1000C0009900C20AC30B71284610C6108316031389
:1000D000981C68280C126C286D286E288312031354
:1000E000061073088400710E8300F00E700E090074
:1000F00007398207013402340434083410342034C0
:100100004034803482078134003441344134C03477
:10011000C134C1340134C134C134403400340134F9
:10012000C134C134003480344034C1348207F034E7
:100130003034D034703430346034E0343034F0341F
:1001400070340034403400349034C0340034C0344F
:10015000F034B03407398207B42801341234223421
:1001600042348234803440346708820701341234C8
:1001700080344034B510CF1908000030E91B01303D
:10018000691B0230691A03306B0782070B2B532B54
:10019000212B662B2A2B132B1C2B662B562B362B35
:1001A0005B2B662B0800802B8D2BE228802B6B2B82
:1001B000782BE228802B962BA02BE228392B262B9C
:1001C000242B662B9801183085000030860083169A
:1001D0000313063086002630850020308C008130E5
:1001E00081000B308E0000309F0083120313053016
:1001F0009F00313090000430920020308400800154
:10020000840A841FFF286C2217240610A723C030FD
:100210008B00193085000C290D290A30E400E50017
:10022000FF30EC0013291429851A4F2901302C24A2
:10023000D3000030D4006030D50014228E018F012D
:100240000C100B197C22C61959210C18492146188B
:1002500021291922013090008E018F010C105623A4
:100260002B2235161030BB000B197C22C6195921E0
:100270000C1C34290C10BB0B3429F030B505E801F7
:100280000B197C22C61959210C18CC23B518BA2099
:1002900040290C100E30E4000730E50008008223EE
:1002A000013090000C1804240B197C22B518BA20D8
:1002B00052292008613A031D89292108031D6B2951
:1002C000CF18122ACF11CF144F100E30E400003097
:1002D000E500E4220F2A013A031D7B29CF11CF103C
:1002E0004F105308D922E4224F080B3903190F2A63
:1002F000C6112B220F2A033A031D122ACF19122AE4
:10030000CF15CF104F100530E4000D30E500E4228A
:100310000F2A033A031D99292108223A031D122AA4
:100320002208CF00CF198329CF1865294F18B1298A
:100330007129013A031DA5292108213A031D122A1A
:100340002208C7002308C800122A2008813A031D8A
:10035000B7292108031D122A4F18122ACF11CF10D6
:100360004F140E30E4000530E500E4220F2A200887
:10037000E13A031DC6292108883A031D122A0530D7
:10038000E4000A30E500CC30EC00122A033A031DE9
:10039000D3292108F039203A031D122A49155308A0
:1003A000D200D501F329013A031DE6292108403A7C
:1003B000031D122A22083F39031D122A230853065F
:1003C000031D122A4914E4223516122A073A031D86
:1003D000032A2108F039031D122A49115308D200BB
:1003E00023081F39D500A21BD516211CA1185517AB
:1003F0002119D51722087F39D4004910A1194914B1
:10040000E4223516122A013A031D122A2108F03976
:10041000103A031D122A49152508D200F029003090
:10042000EB00E422C61108002130572221305F2260
:10043000682A2130572224305F22682A80305722D0
:10044000682A2130572280305F22682A21305722C3
:1004500081305F22682AE330572200305F2200306B
:100460005F2253085F22682AE43057221030551B60
:100470001230D51B13305F2200305F2253085F22F9
:100480005408D51A80385F224910E4225308FB0033
:1004900001303224682AE430572220305F220030B5
:1004A0005F2253085F2255081F395F22442ABC008F
:1004B000C61959214618582AC201C3013C08BD007B
:1004C000A030430784003D088000C206C30A08002C
:1004D00042085F224614080000302C241F3940389F
:1004E000C100BD003D0EBD063D0CBD063D19BD0A57
:1004F0003D0C0318C11708000B11B82318308500F4
:10050000E60A660807390319902A6508E61964089F
:10051000C322EC1F0800E61D0512E619851108002C
:10052000351D982AEA0B080035117830EA000800DA
:10053000670A0339E7000830C3229E2A9F2AA02AAF
:10054000A12A3E08D139BE003E09E8053E08851AB9
:10055000E80468080319B72A3518BD2A3514B511FF
:100560006808E90035150830EA00B5140800670886
:10057000031D08003510B5110800EA0B0800B51579
:100580001030EA00B52ABD006608AA20BE008B1311
:100590003E3085050F3086053D08BE1CD42A9620C6
:1005A0003E0586048B17080082203E0585048B17C4
:1005B0000800BA00F2223808BD003D0E0F39E400F1
:1005C0003D080F39E5000800FF30EB08031DDF3060
:1005D0004918CC30CF18C3304F18C330CF19C330AF
:1005E000EC00080003100830BF00B801B901BA0DD3
:1005F000B80DBF0BFC2A08003830FF22F72A840010
:1006000003300007BD00BD19800030300007BD0079
:10061000BD1B800008001030E4000F30E5000430FE
:10062000EB00E4220800D30A6430530601300319BA
:10063000D3002B225308D92AD30363300319D300E4
:10064000192B1030D5064B2A0230282B0130282BCD
:10065000D5064B220B30D5180C30E5000B30551861
:100660000C30E4001830EB00E42208002030D506FE
:1006700034226308031D562BD51E472B1130E4008E
:100680000B30551B0A30D51B0C30E5004F2B0B30BF
:10069000551B0A30D51B0C30E4001130E500083042
:1006A000EB00E42208002030D50634220030EB00B5
:1006B000E4225308D92A6308031D08008030D51F9F
:1006C0004030551BC030D5063422392B4F18262A0E
:1006D000CF18672B212A00302C24FB00FB0A203086
:1006E0007B0601300319FB00003032247B08D92A35
:1006F00000302C24FB00FB031F300319FB00742B7C
:10070000C91D852BC9111230872BC9150D30E40086
:100710000F30E5000C30EB0008001430C91D10301C
:10072000EB00C919080000302C24D92A02302C24EF
:10073000FB00FB0A7B1AFB037B08E2000230322C31
:1007400002302C24FB00FB03FB1BFB019C2B8316BC
:100750003330920083120430920002302C240F397F
:10076000E2001F30E100620795000C30970008009E
:1007700060080739583E84009F1FC22B6108800023
:10078000E00AC72B9503E10B08008001E00A1F3047
:10079000E1006207950008000C100310EC1B031425
:1007A000EC0D46180800580859075A075B075C0704
:1007B0005D075E075F07BD00BD0CBD0C3D0C1F391A
:1007C000BD006306031908003D08E300351A022C3A
:1007D000551BF32BD51BFD2B3D0C0F39013A031D87
:1007E000013AD400342A04303D02031CBD013D0C03
:1007F000031810381F39D400342ABD0D3D0D7C3943
:10080000D400342A351208000C106B08143A031D6A
:100810000800580859075A075B075C075D075E0721
:100820005F07BD00BD0CBD0C3D0C1F39D92A061059
:10083000C601C50183160313033099006430980084
:1008400083120313D03098000301FF3E031D252CB3
:100850001A081A081A08080083169B001C141A08A4
:10086000831208002C247B06031908007B088316DA
:100870009A001C158B1355309D00AA309D009C14C6
:0C0880008B171C119C18422C83120800DE
:02400E00503F21
:06420000010003000000B4
:104220002034533469346D3470346C346534203444
:104230004D34613475347334203476342E34323452
:1042400046342E3443346134F1346134643461349F
:10425000333430342F34313430342F343034363436
:00000001FF
